:0800000010308A00002D000001
:100080000000000000000000000000000000000070
:1000900003178D018F0110308C0030308E008316D5
:1000A0008C170C15831203130B08F8008B1383169F
:1000B000031755308D00AA308D008C14000000000D
:1000C0008C1860280C117808831203138B040130FC
:1000D00003178D008F018A308C008E0183168C17D8
:1000E0000C15831203130B08F8008B1383160317E8
:1000F00055308D00AA308D008C14000000008C1843
:100100007F280C117808831203138B040230031725
:100110008D008F018C012D308E0083168C170C15ED
:10012000831203130B08F8008B1383160317553043
:100130008D00AA308D008C14000000008C189E28C1
:100140000C117808831203138B048A018201003496
:102A000084011F308305073083169F000230990030
:102A100022309800903083129800A001A10110305C
:102A2000A2003030A3008A30A400A501A6012D30F9
:102A3000A700FF30EF00EF106F08831687008312A6
:102A40008714023083169900223098009030831248
:102A5000980002308316990022309800903083123B
:102A600098000F30F70007308101813084000008A2
:102A7000F0390738800064000008F03977048000DE
:0A2A8000A32564009626412D630093
:022A9E008C1A90
:102AA000532D64004F2D8C1E532D1A088316A00041
:102AB0008312981C612D1A088316A0008312181225
:102AC000181683162008F800831200342808073CE3
:102AD000031D6F2D07300C1E6B2D9900A22D0530A4
:102AE000FC007C08063C0319A22D7C08053C031D54
:102AF0009E2D2830FE006E08F60004300C1E7E2D40
:102B000099006E080C1E822D9900FD016E087D0251
:102B100003189A2D7E08840000088316A0008312F3
:102B20000C1E902D99007E0884000008F606FE0A0F
:102B3000FD0A862D76080C1E9B2D99004F257808DE
:102B4000FC00712D0034B130A8000130EE00662584
:102B50000034F3012830F400F308031DE42D4F2561
:102B60007808F0007008043C0319BA2D4F25780846
:102B7000F000B22D4F257808EE006E08F200F1014A
:102B80006E0871020318D22D7408F5004F257508E0
:102B9000840078088000740884000008F206F40AB3
:102BA000F10AC02D4F257808F206F208031DDF2D2B
:102BB0000130F30006300C1EDB2D9900E32D0530AB
:102BC0000C1EE02D9900AC2D003403306E02003A4B
:102BD0000319502EF1012A08F0007008F1002908AD
:102BE000F0002B30F5000330F4006E087402031877
:102BF000502E7508F50A84000008FA01F2007A08E0
:102C0000F3007508F50A84000008F600F300710867
:102C1000143C03180F2E7108163C03184A2E710835
:102C20001F3C031C4A2EF108031D292E7008033C8B
:102C3000031C292E0310700DF900710DFA0079089C
:102C4000203E8400840A7308800084037208800098
:102C50004A2E700803178D0071088F0072088C00CF
:102C600073088E0083168C170C15831203130B0840
:102C7000F8008B138316031755308D00AA308D0092
:102C80008C14000000008C18432E0C11780883125D
:102C900003138B04F00A0319F10A0230F407F52D2F
:102CA0000730A8000130EE0066250034F0017008FE
:102CB000033C031C8C2EF2017008F1000310700D10
:102CC000F700203E8400840A0008F4008403000812
:102CD000F300700803178D0072088F0073088C00D2
:102CE00074088E0083168C170C15831203130B08BF
:102CF000F8008B138316031755308D00AA308D0012
:102D00008C14000000008C18832E0C11780883129C
:102D100003138B04F00A572E8C2E00342808A900C8
:102D2000FF30A8000230EE0066250034A9252808EF
:102D3000F700313077020319A62E323077020319DB
:102D4000A82E333077020319AA2EAC2EA325AE2E5F
:0E2D5000E525AE2E5626AE2E8E26AE2E003473
:02400E003D3F34
:00000001FF
